:20000000F04C97137EF06A8620B7700001A7007D007A2B0496132A037EE75984F08A069758
:200020001339BDF9C0D660C5202643840327388103273B0E7D0015262B97157F0052962189
:2000400085082705CE80002003CE8800DF16DF1ADF1FDF1C96168B0797187F007A86CF9767
:20006000197EE6A49715397D00152702200739847F81142606868097152027DE1FB770007E
:2000800001A700089C1C260B96038A209703BDFB8B200F9C182602DE16DF1F7D00002B0200
:2000A000DF1AD684C49FCA20D784F77C0039DE1C9C1A2713B7700001A600B77C01089C18F1
:2000C0002602DE16DF1C399684849FD614C1012704D6152A0ED615C508270E7F00158A404E
:2000E0007F00149784B77C00394FB77C018688971539000000000000000000000000000070
:200100000FB77F0EB77F0ACE7F008665A7008644A701865DA702B67E008402270A8620A737
:20012000048614A70520088640A7048635A7058617A703A70697254FA70DA70CA70E8E03C9
:20014000FF7F8F807F8F81CE03FFC6AAE7000926FBCE03FFC6AAE100261053E700E100269A
:20016000096F000926EE6F00200AA600B78F81F78F8020EDB68F8136B68F8036CE8FFFC6B8
:20018000AAE700098C800026F8CE8FFFC6AAE100261153E700E100260A6F00098C800026C2
:2001A000EB2008A60097DBD7DA20EE96DB3696DA364FCEE800A8000826FB36FEE0008C543E
:2001C0004A260DB67D002B087C0000BDE0872004861D971ECE78006F016F03867FA70086C6
:2001E0001DA702863CA701A7038601A7008611A7028643B77A00B77C00B67E0016841C8A16
:20020000C19783B77A0053C4205858D792B67900841C8A419784B77C008617CE8000DF21AF
:20022000DF239725FF87D0FF87D2B787D4CE8800FF8FD0FF8FD2B78FD4BDFA7FBDF827CE32
:200240000055DF7DFE7B1E8C30462605CE7B00200C96002605CEEAF92003CEE545DF53DF16
:200260007FC61EBDF412B6005DF60065C5402602862036BDF3B5BDFDD3B60062BDF2ADBDBE
:20028000F3B5BDFDD3B60062BDF2AD3230A601AA03AA002742CEEABF8D32BDF06A30C605A4
:2002A000BDFC813232323232BDEE7A7D007A2AF8202A5465737420436F6D706C6574654D3C
:2002C000454D4F5259204552524F5220DF7FC60DDE23DF7D7EF412CEEAB28DF0B60066169D
:2002E0008401B77802C5082703BDFB64B67E0084C09751BDFBF47EF8D01B0D0000000001BA
:200300000020000000000002F0030100000000000000000000000000000921D1D1D7D7C588
:20032000C5D2D2D4F4D9F932221B1B7F7F9E9FD0F0B4B6929331217151989833233424357F
:20034000253626372738283929305F2D3D5E7E5C7C09C98787888889892D2D775765457209
:200360005274547959755569496F4F70505B7B5D7D0D0D84848585868609096141735364D1
:20038000446646674768486A4A6B4B6C4C3B2B3A2A40600A0A82828383818190917A5A78F6
:2003A000586343765662426E4E6D4D2C3C2E3E2F3F20201FCA30302E2E0D0D9D941E1E0AA1
:2003C0000A0B0B08080C0CE3402C2CECEBEED9EE39EE3DEEB5ECEBECEBECEBEE50ECEBEC41
:2003E000EBECEBECEBEEB5EE5CEE94ECEBECEBFB60FB5BECEBECEBFB11FB21FB2AFB25FD7E
:20040000AAFD83FDA6F2BEFBA4F482F258F266F272F2AAF460F468F464F46CFCF6FCFBFD5A
:2004200074FD7EECEBF301ECEBF47EFCC6FCD9FB2EFB34FB3BFEB7ECEBFB99ECEBF1AFF30A
:2004400088F388FCC2ECEBECEBECEBFCBEFE67FF55F470FE18FB52ECEBFE8EFB57FD18EC66
:20046000EBECEBECEBECEBECEBECEBFCEBECEBECEBECEBECEBECEBECEBECEBECEBF101ECE1
:20048000EBECEBFCD9FCFFECEBFBFFFCC2FB82FB87F474FE60FB57FB64FB7EECEBFD24EC68
:2004A000EBECEBECEBECEBECEBECEBECEBECEBECEBECEBECEBF486ECEBFB8BEFE3F101EF61
:2004C000D4EFEAEFC9EFF8ECEBECEBECEBECEBECEBECEBECEBECEBECEBECEBECEBECEBECD0
:2004E000EBECEBECEBECEBEFB0EFF139C6049675B77800B678002B0B260286584A97755AB6
:2005000026EC39F67802D7775849CEEB1BBDEE9CC60FD779A6002B1ED677C501270A8161DC
:200520002D06817A2E028020C540270A81402D06817F2702841F4D2A0D81902C097D006719
:200540002B04847F8B309776867D9778CE00019676BDF990860ABDF9A49678271C8602BDEE
:20056000F9A4B678002A1C7A007826F1967981032F037A0079977820D38604BDF9A4B67895
:20058000002BF67F00783936BDF9993216C4F8C198270CD62D2708819026037F002D394D57
:2005A0002A255FBDF9C8847F85602774D651C4C0C140266CD667C40427037EEE2036965572
:2005C000BDF7B2327EF7B2811B2606D6772A029655D651C5402720BDF7B2D6512B01398546
:2005E000602614810D2708810427048103260836CE0007BDF99232BDEEE5DECBE6B3C50125
:20060000260139DFCD7800CEDECDEEA3DF7BBDF9C0D651C1C02603BDF7B2DE7BAD0020DA45
:20062000847F80102B0BCEEBCB48BDEE9CEE006E008B4F7F00787EF48A9667200396674355
:200640008502270486D3200286B5CE00017EF9907F0078B678028801B77802397F0078B695
:200660007E00840126F596838A60B77A0086C8BDF9A49683B77A007EF999F6780037C609B2
:20068000F77800F678002A07F678022A028D0533F77800397F0078C680D77A39DFCD9BCE67
:2006A00097CE96CD890097CDDECD39D6CCC10126037F007839BDFB8B7F0078D6772A0ABD6C
:2006C000F9C07F00784D7EEE20BDF9C07F00784D2BE2856027DE7EF48A9677854026037E6B
:2006E000FD7E7EFDAABDF9D6C520261091552626C6207EF9C89155261DBDF9C05FBDF9C8E0
:2007000081582704817526037EFB578560271ED62A26317EEE2085602709817F260FD62A8F
:20072000260B39D62A2606CEECAB7EEE297D002E270536BDFE6A329A29DE23B7700001A732
:20074000007EEFC936861B8DE43220E10000000000000000000000000000000000000000E8
:20076000000000000000000000000000000000000000000000000000000000000000000079
:20078000000000000000000000000000000000000000000000000000000000000000000059
:2007A0000000000000000000000000000000000096522A0D8404F67802C404112703BDF36F
:2007C000B5BDF0268D517EF151BDF0478D4920F6DE2320F8D6282704D6642B15BDF06E8DAF
:2007E0003620E3BDF0C68D2F20F9BDF0DF8D2820F2BDF06A8D2120CED628DA812609D663B1
:00000001FF
